:10000000B401902AAF21B6000408B8000800AF215F
:10001000B7000408B9000800B600A82184133230E4
:10002000A600A7016A22A00AA50AA201A30100084E
:100030003605A600640000083605A7002606270539
:1000400036060319A20A0319A30A2708A600A40367
:100050000319A5030319A00B1A2822088B2A0408E8
:10006000A2008316861183120930A30003103F20DB
:10007000A20CA30B372803143F2003148B2A031868
:100080004428000086154628861146280030A10025
:10009000C330FA290408A7000610861086108316BC
:1000A0000610861086100F30860583122708B418B4
:1000B00077283A30A1009830FA213330A6008B20FF
:1000C0001330A1008830FA218B206430F9218B2075
:1000D0006430F9212230A6008B20283076200C30A5
:1000E000762006307620B414270877283414A6002A
:1000F000341C85288610033C031C8A288A2007307C
:10010000A100D030FA21031408003414FE3C031976
:100110008B2A8614341C341006140F3086052608EA
:10012000F03986040610A60E34188B283230F921D7
:1001300003140800AF21B600AB21200821040319E5
:100140008B2A80228413360880066400A728A828FA
:10015000A00A0319A10FA52880068B2A6400C420D9
:100160000318AE280B21A8010830A3000C21C420DD
:100170000318A80AAB1EA801A20CA30BB628AB1A41
:10018000A2130C21220808003808840036088417BE
:100190008004841300052B1B3606FF3E0800A401D3
:1001A000A501B5128622D33E0319B5162D3EC63ED3
:1001B0000318DE280A3E031CD228E528F33E031864
:1001C000D228063E031CD2280A3EA2000430A30017
:1001D0000310A40DA50DA30BE8282208A404A9036D
:1001E000031902298622C63E0318FA280A3E031C78
:1001F0000229E528F33E03180229063E031C0229C2
:100200000A3EE528B51E0929A409A509A40A03196F
:10021000A50A24088B2A35172B081F39FF3EA10099
:100220002A08F53E0318A10A351FFA293513A00044
:1002300002302C22FA29B51329080319B517043006
:10024000A800250E282125082821240E282124086D
:100250000F39F63E0318073E0A3E4B29B51329080D
:100260000319B5170530A8002730A300103044212A
:100270000330A300E8304421A30164304421A301EA
:100280000A30442124084B29A2002508A100240893
:10029000A0004E222008A000A8030319B5132908C6
:1002A000031955292802031808002008031DB51357
:1002B000B51B0800303E862A0830A600A700390882
:1002C0008400370835198004FF3A351D8005AC21BC
:1002D000380884003608A821A001A101B5189C2186
:1002E0003808840000083605FF3EA00DA10DB51C9E
:1002F0009C21A60B6E29270835180E2A20088B2A68
:100300000830A60035180E22390884003708351940
:10031000A321351DA521380884003609AC213808F1
:100320008400A10CA00C00083604031C36068000D3
:100330009C21A60B8F298B2A390884003708800658
:100340000000800608008004AB29FF3A8005AC2934
:10035000841780048B2AFF3A841780058B2AA80013
:100360000630A8190730840001308A0028080739B0
:100370008207013402340434083410342034403409
:100380008034A000A00DA00DA00D3830A005813054
:1003900020049F000030A1003230FA211F151F19E0
:1003A000CF291E08A10083161E088B2A03178D0073
:1003B00083168C130C1483120C088B2A03178C00E1
:1003C00083168C130C1555308D00AA308D008C14BB
:1003D0008C18E8290C118B2AA301A200FF30A20778
:1003E000031CA307031C8B2A0330A100DF30FA2172
:1003F000EE29A101E83EA000A109FC30031C032A5C
:10040000A0070318002AA0076400A10F002A2018E3
:10041000092AA01C0D2A00000D2A0800A400A20130
:10042000A301162AA10CA00CA20DA30DFF3E0318D8
:10043000122A240824222208A0042308A104200848
:1004400008000310A00DA10DFF3E0318212A20086B
:100450008B2A0310A10CA00CFF3E0318292A2008A8
:100460008B2AA20003303E2AA301A20001303E2ABB
:10047000A20006303E2AA20004303E2AA80023082B
:100480002102031D452A22082002043003180130EE
:10049000031902302805031DFF308B2A1030A600F7
:1004A000A501A401210DA40DA50D2208A402230875
:1004B000031C230FA5020318642A2208A40723089B
:1004C0000318230FA5070310A00DA10DA60B522A98
:1004D00020088B2A1030A800A101A001A70CA60CAF
:1004E000031C782A2208A00723080318230FA1075A
:1004F000A10CA00CA50CA40CA80B6E2A24088B2A16
:10050000A009A109A00A0319A10A08008400310862
:100510008A003008820083130313831264000800EA
:100520000330A300E8308A01ED21831604308600F1
:100530001F308500FC3087008312831684309F00B3
:10054000831281309F0064008A110A12071EAF2AAD
:1005500064008A110A12071A6C2F8A01A32AFE303E
:100560008A014B2001308A014B2043308A014B2005
:1005700061308A014B206C308A014B2069308A013E
:100580004B2062308A014B2072308A014B2061304F
:100590008A014B2063308A014B2069308A014B204D
:1005A0006F308A014B206E308A014B2043308A0124
:1005B000302061308A0130206C308A01302069306F
:1005C0008A01302062308A01302072308A01302066
:1005D00061308A01302063308A01302069308A011D
:1005E00030206F308A0130206E308A013020203078
:1005F0008A0130202D308A01302020308A013020BD
:1006000065308A0130206E308A01302074308A01D2
:10061000302072308A01302061308A0130207230FF
:100620008A01302020308A01302076308A01302043
:1006300061308A0130206C308A0130206F308A01AD
:10064000302072308A01302065308A0130207330CA
:100650008A0130200A308A0130200D308A01302092
:1006600043308A0130206F308A0130206D308A019A
:10067000302070308A01302065308A0130206E30A1
:100680008A01302073308A01302061308A013020A5
:1006900063308A01302069308A0130206F308A014E
:1006A00030206E308A01302020308A0130205430D2
:1006B0008A01302065308A0130206D308A01302077
:1006C00070308A0130202B308A0130203A308A0184
:1006D00030200A308A0130200D308A013020053068
:1006E000B8002030B600BC30AA004030AB0001306A
:1006F000A900AE30B000B1018A01CF20F90001306D
:10070000A9007908A400A5012F30B000B1018A0129
:100710001B210A308A0130200D308A013020FE3042
:100720008A014B20C0308A014B2054308A014B2073
:1007300065308A014B206D308A014B2070308A0170
:100740004B2020308A014B202B308A014B20013076
:10075000A9007908A400A5014A30B000B1018A01BE
:100760001B21031701308D00031379088A01DE2154
:100770000330A300E8308A01ED21FE308A014B20CE
:1007800001308A014B2043308A014B2061308A01BD
:100790004B206C308A014B2069308A014B2062303B
:1007A0008A014B2072308A014B2061308A014B2034
:1007B00063308A014B2069308A014B206F308A01F7
:1007C0004B206E308A014B2043308A0130206F303D
:1007D0008A0130206D308A01302070308A0130204B
:1007E00065308A0130206E308A01302073308A01F2
:1007F000302061308A01302063308A013020693036
:100800008A0130206F308A0130206E308A0130201A
:1008100020308A01302054308A01302065308A012E
:1008200030206D308A01302070308A0130202D3028
:100830008A0130203A308A0130200A308A01302083
:100840000D308A0130200530B8002030B600BC30B1
:10085000AA004030AB000130A900AE30B000B101B9
:100860008A01CF20F9000130A9007908A400A50170
:100870002F30B000B1018A011B210A308A013020DB
:100880000D308A013020FE308A014B20C0308A01B1
:100890004B2054308A014B2065308A014B206D304B
:1008A0008A014B2070308A014B2020308A014B2076
:1008B0002D308A014B200130A9007908A400A50140
:1008C0004A30B000B1018A011B21031702308D00AC
:1008D000031379088A01DE210330A300E8308A017E
:1008E000ED21FE308A014B2001308A014B2043303C
:1008F0008A014B2061308A014B206C308A014B20E9
:1009000069308A014B2062308A014B2072308A01A3
:100910004B2061308A014B2063308A014B206930C3
:100920008A014B206F308A014B206E308A014B20A8
:1009300043308A0130206F308A0130206D308A01C7
:10094000302070308A01302065308A0130206E30CE
:100950008A01302073308A01302061308A013020D2
:1009600063308A01302069308A0130206F308A017B
:1009700030206E308A01302020308A01302048300B
:100980008A01302075308A0130206D308A01302094
:100990002B308A0130203A308A0130200A308A0117
:1009A00030200D308A0130200530B8002030B600EC
:1009B000BC30AA004030AB000130A900AE30B0001E
:1009C000B1018A01CF20F9000130A9007908A40003
:1009D000A5012F30B000B1018A011B210A308A0124
:1009E00030200D308A013020FE308A014B20C0308B
:1009F0008A014B2048308A014B2075308A014B20F8
:100A00006D308A014B2020308A014B202B308A0127
:100A10004B200130A9007908A400A5014A30B0009C
:100A2000B1018A011B21031703308D0003137908DC
:100A30008A01DE210330A300E8308A01ED21FE3077
:100A40008A014B2001308A014B2043308A014B2020
:100A500061308A014B206C308A014B2069308A0159
:100A60004B2062308A014B2072308A014B2061306A
:100A70008A014B2063308A014B2069308A014B2068
:100A80006F308A014B206E308A014B2043308A013F
:100A900030206F308A0130206D308A013020703074
:100AA0008A01302065308A0130206E308A01302082
:100AB00073308A01302061308A01302063308A012E
:100AC000302069308A0130206F308A0130206E304A
:100AD0008A01302020308A01302048308A013020BD
:100AE00075308A0130206D308A0130202D308A0126
:100AF00030203A308A0130200A308A0130200D300F
:100B00008A0130200530B8002030B600BC30AA0081
:100B10004030AB000130A900AE30B000B1018A0115
:100B2000CF20F9000130A9007908A400A5012F30D9
:100B3000B000B1018A011B210A308A0130200D303A
:100B40008A013020FE308A014B20C0308A014B20C0
:100B500048308A014B2075308A014B206D308A0164
:100B60004B2020308A014B202D308A014B20013050
:100B7000A9007908A400A5014A30B000B1018A019A
:100B80001B21031704308D00031379088A01DE212D
:100B90000330A300E8308A01ED21FE308A014B20AA
:100BA00001308A014B2043308A014B2061308A0199
:100BB0004B206C308A014B2069308A014B20623017
:100BC0008A014B2072308A014B2061308A014B2010
:100BD00063308A014B2069308A014B206F308A01D3
:100BE0004B206E308A014B2043308A0130206F3019
:100BF0008A0130206D308A01302070308A01302027
:100C000065308A0130206E308A01302073308A01CD
:100C1000302061308A01302063308A013020693011
:100C20008A0130206F308A0130206E308A013020F6
:100C300020308A01302050308A01302072308A0101
:100C4000302065308A01302073308A0130207330C3
:100C50008A0130202B308A0130203A308A0130203E
:100C60000A308A0130200D308A0130200530B8006A
:100C70002030B600BC30AA004030AB000130A900E3
:100C8000AE30B000B1018A01CF20F9000130A900D7
:100C90007908A400A5012F30B000B1018A011B2101
:100CA0000A308A0130200D308A013020FE308A015E
:100CB0004B20C0308A014B2050308A014B207230CB
:100CC0008A014B2065308A014B2073308A014B200A
:100CD00073308A014B2020308A014B202B308A014F
:100CE0004B200130A9007908A400A5014A30B000CA
:100CF000B1018A011B21031705308D000313790808
:100D00008A01DE210330A300E8308A01ED21FE30A4
:100D10008A014B2001308A014B2043308A014B204D
:100D200061308A014B206C308A014B2069308A0186
:100D30004B2062308A014B2072308A014B20613097
:100D40008A014B2063308A014B2069308A014B2095
:100D50006F308A014B206E308A014B2043308A016C
:100D600030206F308A0130206D308A0130207030A1
:100D70008A01302065308A0130206E308A013020AF
:100D800073308A01302061308A01302063308A015B
:100D9000302069308A0130206F308A0130206E3077
:100DA0008A01302020308A01302050308A013020E2
:100DB00072308A01302065308A01302073308A0118
:100DC000302073308A0130202D308A0130203A30B3
:100DD0008A0130200A308A0130200D308A0130200B
:100DE0000530B8002030B600BC30AA004030AB005F
:100DF0000130A900AE30B000B1018A01CF20F90066
:100E00000130A9007908A400A5012F30B000B1017C
:100E10008A011B210A308A0130200D308A013020DE
:100E2000FE308A014B20C0308A014B2050308A01AD
:100E30004B2072308A014B2065308A014B20733081
:100E40008A014B2073308A014B2020308A014B20CD
:100E50002D308A014B200130A9007908A400A5019A
:100E60004A30B000B1018A011B21031706308D0002
:100E7000031379088A01DE210330A300E8308A01D8
:100E8000ED21FE308A014B2001308A014B20503089
:100E90008A014B2075308A014B206C308A014B202F
:100EA00073308A014B2061308A014B2072308A01F5
:100EB0004B2020308A014B2052308A014B20653074
:100EC0008A014B2073308A014B2065308A014B2008
:100ED00074308A014B200800FE308A014B2001301B
:100EE0008A014B2020308A014B2050308A014B2050
:100EF00049308A014B2043308A014B202D308A0132
:100F00004B2057308A014B2058308A014B2020302B
:100F10008A014B2053308A014B2054308A014B20E8
:100F200041308A014B2054308A014B2049308A01DC
:100F30004B204F308A014B204E308A014B2020300D
:100F40008A014B20FE308A014B20C0308A014B20A1
:100F500045308A014B2041308A014B2033308A01D1
:100F60004B2043308A014B204E308A014B204F30BA
:100F70008A014B2020308A014B2020308A014B20EF
:100F800020308A014B2057308A014B2058308A018B
:100F90004B205F308A014B2041308A014B2050307A
:100FA0008A014B2052308A014B2053308A014B205A
:100FB0000B30A300B8308A01ED2187168316871203
:100FC0000F3083128A0102200E308A010720B501FA
:100FD0000C30A000A1018A0180210230A000A101F3
:100FE0008A0180218712831687128312F701F40188
:100FF000F501C201C3018316A101831200308A01E9
:10100000C121C0002108C10001308A01C121BA00FC
:101010002108BB00CA30A2000830A30006308400BB
:1010200004308A010C208316A200013083128A0149
:10103000D621F10002308A01D621F00003308A0166
:10104000D621ED0004308A01D621EC0005308A015A
:10105000D621EF0006308A01D621EE008A150A1249
:101060005C218A150A1292217108D0070318D10A4F
:101070007008D002031CD1038A150A12B9218A15FF
:101080000A12E4218A150A120F228A150A126C220A
:101090008A150A12EA228A150A1208238A150A12E8
:1010A00018238A150A125C238A150A128523640004
:1010B0008A150A12871DFE2C64008A150A12071E63
:1010C000722D5008A0005108A1000130A30000308B
:1010D0008A0131228A150A12031DF62B5008A0003E
:1010E0005108A1000130A30000308A013B228A157B
:1010F0000A12031D7A2C8A150A12C9238A150A12AC
:10110000D8238A150A12E723C20A0319C30A420820
:10111000A0004308A100A30104308A0138228A11EB
:101120000A12031DFE2F0330A9003E08A4003F0849
:10113000A5002F30B000B1018A012E212C308A0188
:1011400030200330A9004A08A4004B08A5002F3026
:10115000B000B1018A012E212C308A0130200330E9
:10116000A9007408A400A5012F30B000B1018A01C4
:101170002E212C308A0130200330A9005008A40011
:101180005108A5002F30B000B1018A012E212C306A
:101190008A0130200430A9004408A4004508A500B5
:1011A0002F30B000B1018A012E212C308A0130206D
:1011B0000230A9007608A400A5012F30B000B101CB
:1011C0008A012E212C308A0130202E308A013020D5
:1011D0002E308A0130202C308A0130202E308A01B6
:1011E00030202E308A0130202C308A0130202E30E1
:1011F0008A0130202E308A0130202A308A013020A6
:101200000330A9004C08A4004D08A5002F30B00001
:10121000B1018A012E212C308A0130200330A9002F
:101220007508A400A5012F30B000B1018A012E215C
:101230002C308A0130200330A90083162008831245
:10124000A400A5012F30B000B1018A012E212A305F
:101250008A0130202A308A0130200230A9007C081F
:10126000A400A5012F30B000B1018A012E212E303B
:101270008A013020A9017E08A400A5012F30B0000A
:10128000B1018A012E210A308A0130200D308A01F5
:101290003020C201C3018316A10A64002D3021024F
:1012A0008A110A128312031CFE2FF401F501831622
:1012B000A10183128A01FE2F8716831687120F3031
:1012C00083128A0102200E308A010720B501EE3018
:1012D000A000A1018A018021871283168712831240
:1012E0008716831687120F3083128A0102200E3070
:1012F0008A010720B501AA30A000A1018A0180213E
:101300000F308A0102200E308A0107200130B5001B
:101310008A015C21CE002108CF0087128316871234
:10132000831208004E08A0004F08A100A301C83096
:101330008A013B228A150A12031DAB294E08A00020
:101340004F08A100A301C9308A0131228A150A126F
:10135000031DB429080000304E07D00001300318E7
:10136000013E4F07D10008004E08D0004F08D100C1
:10137000080000305002B2000130031C013E51024F
:10138000B300330C320CFC0000305002B2000130CC
:10139000031C013E5102B3003208A0003308A10033
:1013A0000230A200A3018A014E222408B2002508BF
:1013B000B3003208A6003308A7000530A200A3013D
:1013C0008A016A22FE0008005008003CB200510861
:1013D000031C013E013CB300330C320CFD005008ED
:1013E000003CB2005108031C013E013CB30032082E
:1013F000A0003308A1000230A200A3018A014E22FE
:101400002408B2002508B3003208A6003308A7005C
:101410000530A200A3018A016A22FF000800510CD6
:10142000500CF2005008A0005108A1000230A200A8
:10143000A3018A014E222408B2002508B300320815
:10144000A6003308A7000530A200A3018A016A2282
:10145000F30092307207B200FF300318013EB30070
:101460003208A6003308A7000A30A200A3018A01AF
:101470006A22BC002508BD003C08A0003D08A10070
:101480000530A200A3018A014E22B2002108B30058
:101490003208A6003308A7000930A200A3018A0180
:1014A0006A22B2002508B3003208A0003308A10068
:1014B0000A30A200A3018A014E228316A000640014
:1014C0000530831273028A150A120318682A08006D
:1014D0008316A00A831208003A08A6003B08A7005A
:1014E0003230A200A3018A016A22B2002508B300AB
:1014F0003208A0003308A100FF30A2000330A3008F
:101500008A014E22C6002108C7003A08A6003B08FF
:10151000A7003230A200A3018A016A22B200250886
:10152000B3003208A0003308A100FF30A20003304E
:10153000A3008A014E222408C8002508C9004608D5
:10154000A6004708A700E830A2000330A3008A01E4
:101550006A22B2002508B3004808B20749080318F8
:10156000013EB3073208A0003308A100F430A20006
:101570000130A3008A014E22B2002108B3001030CE
:10158000B2020030031C013EB3023208A600330849
:10159000A7006430A200A3018A016A22B2002508D4
:1015A000B3003208A0003308A1003E30A200A3011E
:1015B0008A014E22F6006D08F6076C08F6026400F8
:1015C000643076028A150A120318E72A080063308D
:1015D000F600080007108316071083128710831681
:1015E000871083126430A000A10109308A019A207B
:1015F0000A308A01022009308A0107200230B50032
:101600008A015C21F8000714831607108312080072
:1016100020307807C40003300318013EC5006F086E
:10162000C4070318C50A6E08C402031CC5030800DA
:10163000831622088312A600A701A330A200A301EB
:101640008A016A22B2002508B3003208A0003308DC
:10165000A1006430A200A3018A014E22B200210839
:10166000B30001303202CA000030031C013E3302D5
:10167000CB00831622088312A600A701A330A20084
:10168000A3018A016A22B2002508B3003208A00033
:101690003308A1006430A200A3018A014E2224086D
:1016A000FA00640034307A028A150A120318582BA3
:1016B000CA0A0319CB0A08002430A600A701400873
:1016C000A2004108A3008A016A22B2002508B300E3
:1016D0003208A0003308A1006630A200A3018A01ED
:1016E0004E22BE002108BF003E08A0003F08A10016
:1016F0000130A30068308A0131228A150A12031DC5
:10170000822B0800BE01BF01080083162208831245
:10171000A600A7016730A200A3018A016A22B200D5
:101720002508B3003208A0003308A1006430A200ED
:10173000A3018A014E22B2002108B3000130320217
:10174000CC000030031C013E3302CD00831622087A
:101750008312A600A7016730A200A3018A016A22B2
:10176000B2002508B3003208A0003308A10064309D
:10177000A200A3018A014E222408FB006400343039
:101780007B028A150A120318C52BCC0A0319CD0A4D
:1017900008004A08A0004B08A10077088A013422FB
:1017A0008A150A12031DD52B08004A08F700080005
:1017B0004A08A0004B08A10074088A0134228A1547
:1017C0000A12031DE42B08004A08F40008004C0824
:1017D000A0004D08A10075088A0134228A150A125A
:1017E000031DF32B08004C08F5000800FE308A01A9
:1017F0004B2001308A014B202B308A014B200230D4
:10180000A9007C08A400A5014A30B000B1018A01FA
:101810002E212E308A014B20A9017E08A400A501AB
:101820004A30B000B1018A012E21DF308A014B20FD
:1018300043308A014B2020308A014B2020308A011E
:101840004B2020308A014B2020308A014B2002306F
:10185000A9007608A400A5014A30B000B1018A01B0
:101860002E2125308A014B2052308A014B204830EE
:101870008A014B20FE308A014B20C0308A014B2068
:1018800057308A014B2069308A014B206E308A0123
:101890004B2064308A014B2020308A014B200330DA
:1018A000A9004A08A4004B08A5004A30B000B101C5
:1018B0008A012E214B308A014B206D308A014B204A
:1018C00068308A014B2020308A014B200330A90068
:1018D0003E08A4003F08A5004A30B000B1018A01CB
:1018E0002E21DF308A014B200A308A01EC218A1533
:1018F0000A127B28FE308A014B2001308A014B20DE
:101900002D308A014B200230A9007D08A400A501DA
:101910004A30B000B1018A012E212E308A014B20BD
:10192000A9017F08A400A5014A30B000B1018A01D5
:101930002E21DF308A014B2043308A014B2020309A
:101940008A014B2020308A014B2020308A014B2015
:1019500020308A014B200230A9007608A400A5019E
:101960004A30B000B1018A012E2125308A014B2076
:1019700052308A014B2048308A014B20FE308A01C8
:101980004B20C0308A014B2057308A014B206930F0
:101990008A014B206E308A014B2064308A014B2033
:1019A00020308A014B200330A9004A08A4004B08CC
:1019B000A5004A30B000B1018A012E214B308A01C6
:1019C0004B206D308A014B2068308A014B2020303B
:1019D0008A014B200330A9003E08A4003F08A5005F
:1019E0004A30B000B1018A012E21DF308A014B203C
:1019F0000A308A01EC218A150A127B28FE308A01FE
:101A00004B2001308A014B2057308A014B2069302E
:101A10008A014B206E308A014B2064308A014B20B2
:101A200020308A014B2047308A014B2075308A01D3
:101A30004B2073308A014B2074308A014B202030B8
:101A40008A014B200330A9007408A400A5014A3084
:101A5000B000B1018A012E214B308A014B206D303C
:101A60008A014B2068308A014B20FE308A014B20CE
:101A7000C0308A014B2057308A014B2069308A01DF
:101A80004B206E308A014B2064308A014B2020307D
:101A90008A014B204D308A014B2061308A014B2056
:101AA00078308A014B2020308A014B2020308A0177
:101AB0004B200330A9007708A400A5014A30B000EC
:101AC000B1018A012E214B308A014B206D308A01F1
:101AD0004B2068308A014B200A308A01EC218A159C
:101AE0000A127B28FE308A014B2001308A014B20EC
:101AF00050308A014B2072308A014B2065308A01B8
:101B00004B2073308A014B2073308A014B20753093
:101B10008A014B2072308A014B2065308A014B20AC
:101B200020308A014B200430A9004408A400450855
:101B3000A5004A30B000B1018A012E2168308A0127
:101B40004B2050308A014B2061308A014B20FE30FF
:101B50008A014B20C0308A014B2020308A014B2063
:101B600020308A014B2020308A014B2020308A010E
:101B70004B2020308A014B2020308A014B2020301E
:101B80008A014B2020308A014B2020308A014B20D3
:101B900020308A014B2020308A014B2020308A01DE
:101BA0004B2020308A014B2020308A014B202030EE
:101BB0008A014B2020308A014B200A308A01EC2117
:061BC0008A150A127B28C1
:02400E00753DFE
:00000001FF
